Help required in identifying the admin groups for a IT Resource

I would like to pick up the user details of the members in the admin groups of a particular IT resource.
Can anyone help me in this regard..???
Thanks in advance

If you can replace <SMALLIMAGE with <IMG then I am not
sure why you couldn't include the SRC="charcothip.jpg" with the
<IMG portion?
How are you replacing it currently? Could you store the
replacement string in a variable and use it instead.
var replacementString:String = "<IMG
SRC=\"charcothip.jpg\"";
Then you could do something like this (assume the myStr holds
the XML String):
var myArr:Array = new Array();
myArr = myStr.split("<SMALLIMAGE");
myStr = myArr.join(replacementString);
Obviously, this will only work if you are replacing all of
the <SMALLIMAGE pieces with the same image. If not then you
could use the following:
var searchFor:String = "<SMALLIMAGE";
var newString:String = myStr.substring(0,
myStr.indexOf(searchFor));
newString += replacementString;
newString +=
myStr.substr(myStr.indexOf(searchFor)+searchFor.length);
You can keep the width and height attributes since Flash will
recognize those when rendering the HTML.
Tim

Similar Messages

  • How can identify the default currency for a customer?

    How can identify the default currency for a customer?
    I know that this is being determined when you create a sales order for a particular customer, for example, so I could break this process open and find out what it uses. But I thought it worth asking in this forum first.
    Blue

    Hi Gary,
    As per my understanding of your question I am replying , If you are looking some thing else then I request you to please elaborate your query.
    If you see the BP sales area data in transaction BP, In billing tab you maintain the currency for a customer which is default currency when you create a sales order.
    <b>Reward points if it helps!!</b>
    Best regards,
    Vikash

  • We have a requirement to print the w2 forms for employees using java application, how can i implement this. Please give some suggestion.

    We have a requirement to print the w2 forms for employees using java application, how can i implement this. Please give some suggestion.

    Anyone any ideas to help please?

  • Help required to recognize the correct language import package

    Hi friends,
    I am trying to import ukranian(UK) language to SAP system using SMLT transaction.Please help me to identify the correct 'language import package'
    from the DVD dump.I cannot recognize the correct DVD .I am not clear how do I realize the exact package from the DVD dump.Kindly help me.
    Regards,
    Syam krishnan

    Hi Syam
    Please refer the TWO notes for clarity
    Note 97476 - Language availability R/3 4.0x - 4.7x, ECC500
    Note 517310 - Ukrainian language import has been filled w/ Russian
    Cheers,
    Shyam

  • The employee grouping for account determination

    Dear experts!
    Now, I'm getting some issues about The employee grouping for account determination.
    - The first, when I define Employee grouping for account determination, after that I want to know How do I can assign Employee to Employee grouping for account determination.
    - Second, where is I can assign employee group, employee subgroup to Employee grouping for account determination?
    Help me, please!
    Regards Huy!

    First you go to Employee grouping for account determination and make two groups for two Company codes or EE Groups or EE subgroups Etc then assign to company codes In the Standard feature PPMOD Now in the table where you assign Symbolic to GL accounts you assign same symbolic with different groups like this.
    Example:
    Symolic A/C            EE Group for acc determination                                                GL
    001                                    1                                                                                2010201
    001                                    2                                                                               2010202
    Regards.
    Muhammad Afrasyab

  • I suspect a spy app on my iphone 4 that somebody watching my calls/ voice conversation. Can somebody help me to identify the app and how to remove it?

    I suspect a spy app on my iphone 4 that somebody watching my calls/ voice conversation. Can somebody help me to identify the app and how to remove it?

    No spy app can be installed on iphone which is not jailbroken.
    For example iKeyMonitor iPhone spy can not be installed without jailbroken.
    http://ikeymonitor.com

  • Adding responsibility objects for the Notification Groups for a PA

    Hi Gurus,
    I am supposed to add responsibility objects for the notiifcation groups for a PA.. Could you please confirm the steps I am planning to follow
    1. Find out the Workflow
    2. Add the responsibilities objects ( Where can Add  those ( in the workflow or in Org Management?)
    3. Edit the rule to point to that PA..
    I am new to workflows ..points are assured for the help

    Just write your own composite Icon class:
    public class CompositeIcon implements Icon
      private Icon icon1;
      private Icon icon2;
      public CompositeIcon(Icon icon1, Icon icon2)
        this.icon1 = icon1;
        this.icon2 = icon2;
      public int getIconHeight()
        return Math.max(icon1.getIconHeight(), icon2.getIconHeight());
      public int getIconWidth()
        return icon1.getIconWidth() + icon2.getIconWidth();
      public void paintIcon(Component c, Graphics g, int x, int y)
        icon1.paintIcon(c, g, x, y);
        icon2.paintIcon(c, g, x + icon1.getIconWidth, y);
    }Hopefully a slightly more reusable solution. You could write all sorts of different layouts in this way.
    Hope this helps.

  • Acrobat on my new computer is requiring permission from the admin. I am the admin however i dont know how to give myself permission

    Acrobat on my new computer is requiring permission from the admin. I am the admin however i dont know how to give myself permission

    Hi ericr31731540,
    Could you please let me know what version of OS are you using.
    You might need to repair disk permissions.
    Also, please tell me when does Acrobat asks for admin access and what exactly is the message.
    Hope to hear from you.
    Regards,
    Anubha

  • Unable to get the admin object for the CsContainerAdmin service

    Hi,
    On AIX, we deployed XIR2 SP2 --> XIR2 SP3 --> SP3 Productivity Pack.
    The Conection server does show up on the server list in the CMC, but on trying to access this server, it throws an error" Unable to get the admin object for the CsContainerAdmin service"
    Tried to manually create another Connection server, same result.
    Is this an issue that is addressed by a later FP?
    Thanks in advance
    Rajesh Jayakumar

    Hi Rajesh,
    Were you able to resolve this issue? I am facing the same issue with almost every BOE 11.5 SP3 server on Windows.
    For example, the Input file server says this -
    "Unable to get the admin object for the FileServerAdmin service for server Input.BOCMSMSGT1.fileserver".
    Getting the same error on WebI Report Server as well -
    There was an error while retrieving data from the server: Unable to get the admin object for the WebiServerAdmin service for server BOPROCENG1.Web_IntelligenceReportServer.webiserver
    Thanks,
    Sarang
    Edited by: Sarang Deshpande on Sep 26, 2008 3:08 PM

  • Can anyone help me with getting the best setting for me system

    can anyone help me with getting the best setting for me system on cpufan it says my temp is 38c but on corecentre it says 42c can anyone help get my system overclocked any more but keeping it stable as well thanx in advance for the help  

    my corecenter temp sometimes says im at 60 cel at idle....and i have the most recent update...i would rely on speedfan for temp control...core center seems to always read 3 degrees higher than speedfan on my pc....
    i wouldnt be too concerned...those temps are pretty low to begin with.

  • Please help me ,i forgot the synchronising password for my mac pro lion backup disk

    please help me ,i forgot the synchronising password for my mac pro lion backup disk

    If the backup volume is encrypted, and you forgot the password, then you'll have to erase the volume and start a new backup. There's no way to recover the password.

  • Experiencing extreme slowness of the Admin console for any function in Weblogic 12.1.1.

    Experiencing extreme slowness of the Admin console for any function in Weblogic 12.1.1. 
    Configuration is Admin server plus 28 JMS servers - no nodemanager - all on the same server. 
    When I bring up Admin console alone response is quick but bringing up JMS servers one by one will slow it down. 
    I did not experience this problem when this configuration was in Weblogic 9. 
    Memory configuration is -Xms4g, -Xmx4g. 
    Any ideas what else I should check ?
    Thanks.

    Hi,
    Collect multiple thread dump at the interval of 10 sec and check what the threads are doing .
    Thread dumps will give you some information about why there is a slowness .
    Ways to collect thread dumps
    Thread dumps & Ways to take thread dumps - weblogicexpert
    Hope it helps

  • How to get the screen groups for the screen field which are on selectionscn

    hiiii Experts,
                   How to know the screen groups for the screen field which are on selection screen.
    Thanks and regards,
    kasyap

         NAME                                             PNPABKRS-LOW
            GROUP1                                             SEL
            GROUP2                                             DBS
            GROUP3                                             LOW
            GROUP4                                             180
    to get this use this:
    AT SELECTION-SCREEN OUTPUT.
      LOOP AT SCREEN.
        if screen-name CS 'ABKRS'.
          BREAK-POINT.
        endif.
      ENDLOOP.

  • How to dump block and identify the bytes stored for each column

    SQL> select header_file, header_block
    2 from dba_segments
    3 where segment_name = 'APARTMENTS';
    HEADER_FIL HEADER_BLO
    4 1692
    1 row selected.
    SQL> alter system dump datafile 4 block 1693;
    Statement processed.
    How can I see the dump block and identify the bytes stored for each column?
    tab 0, row 0, @0x73b
    tl: 125 fb: H-FL lb: 0x1 cc: 4
    col 0: [25]
    52 65 64 77 6f 6f 64 20 53 68 6f 72 65 73 20 41 70 61 72 74 6d 65 6e 74 73
    col 1: [20] 00 54 00 01 02 08 00 00 00 01 00 00 00 01 00 00 00 00 1b 8d
    col 2: [53]
    00 54 00 01 02 0c 00 00 00 01 00 00 00 01 00 00 00 00 1b 8e 00 21 09 00 00
    00 00 00 00 11 00 00 00 00 00 01 45 6d 65 72 67 65 6e 63 79 20 44 65 74 61
    69 6c 73
    col 3: [20] 00 54 00 01 01 08 00 00 00 01 00 00 00 01 00 00 00 00 1b 8f

    SQL> select header_file, header_block
    2 from dba_segments
    3 where segment_name = 'APARTMENTS';
    HEADER_FIL HEADER_BLO
    4 1692
    1 row selected.
    SQL> alter system dump datafile 4 block 1693;
    Statement processed.
    How can I see the dump block and identify the bytes stored for each column?
    tab 0, row 0, @0x73b
    tl: 125 fb: H-FL lb: 0x1 cc: 4
    col 0: [25]
    52 65 64 77 6f 6f 64 20 53 68 6f 72 65 73 20 41 70 61 72 74 6d 65 6e 74 73
    col 1: [20] 00 54 00 01 02 08 00 00 00 01 00 00 00 01 00 00 00 00 1b 8d
    col 2: [53]
    00 54 00 01 02 0c 00 00 00 01 00 00 00 01 00 00 00 00 1b 8e 00 21 09 00 00
    00 00 00 00 11 00 00 00 00 00 01 45 6d 65 72 67 65 6e 63 79 20 44 65 74 61
    69 6c 73
    col 3: [20] 00 54 00 01 01 08 00 00 00 01 00 00 00 01 00 00 00 00 1b 8f

  • DPM 2012 still requires put end users into local admin groups for the purpose of end user data recovery?

    On client computers that are protected by DPM 2010 and prior versions, you had to put the end users account in the local administrators group. If you did not add the end user account to the local administrators group you would get this error after opening
    the recovery tab in the DPM client: “DPM found no recovery points which you are authorized to restore on the specified DPM server. You can restore only those recovery points for which you were an administrator at the time the
    backup was taken. To restore other recovery points, contact your DPM administrator, or attempt to restore from another DPM.”  This is not ideal on many networks because the end users are not allowed to have local administrator access.
    Ths fix to this was included in hotfix 2465832 found here: http://support.microsoft.com/kb/2465832.
    This hotfix (a hotfix rollup package for DPM 2010) resolves other issues with DPM 2010 as well. You can find the full list of what this hotfix corrects on that link.
    One would think this issue should have been resolved in DPM 2012, however I am encountering the same exact issue, had to include end-users into the workstation local admin group before they can search for recovery points on the DPM server. This is not acceptable
    practice.
    Is there a new hotfix for the same issue on DPM 2012? I am hesitated to apply KB2465832 since it also includes many other fixes for DPM 2010, which may not appicable for version 2012.
    Please help.
    Thanks,

    This is a hands off solution to allow all users that use a machine to be able to restore their own files.
    1) Make these two cmd files and save them in c:\temp
    2) Using windows scheduler – schedule addperms.cmd to run daily – any new users that log onto the machine will automatically be able to restore their own files.
    <addperms.cmd>
    Cmd.exe /v /c c:\temp\addreg.cmd
    <addreg.cmd>
    set users=
    echo Windows Registry Editor Version 5.00>c:\temp\perms.reg
    echo [HKEY_LOCAL_MACHINE\SOFTWARE\Microsoft\Microsoft Data Protection Manager\Agent\ClientProtection]>>c:\temp\perms.reg
    FOR /F "Tokens=*" %%n IN ('dir c:\users\*. /b') do set users=!users!%Userdomain%\\%%n,
    echo "ClientOwners"=^"%users%%Userdomain%\\bogususer^">>c:\temp\perms.reg
    REG IMPORT c:\temp\perms.reg
    Del c:\temp\perms.reg
    Please remember to click “Mark as Answer” on the post that helps you, and to click “Unmark as Answer” if a marked post does not actually answer your question. This can be beneficial to other community members reading the thread. Regards, Mike J. [MSFT] This
    posting is provided "AS IS" with no warranties, and confers no rights.
    That's a good one! Thanks for that.
    I've been scripting on KIX for some time, so here is mine, hope it helps to someone... (it's probably not the best, but it works)
    ========================================================================
    $RC=setoption("WOW64AlternateRegView","on") 
    $DPMkey = "HKEY_LOCAL_MACHINE\SOFTWARE\Microsoft\Microsoft Data Protection Manager\Agent\ClientProtection"
    $uservariable = "%userdomain%\%username%"
    If KeyExist ($DPMkey)
    $Userstring=ReadValue($DPMkey, "ClientOwners")
    If $Userstring == ""
    WriteValue($DPMkey,"ClientOwners", $uservariable, "REG_MULTI_SZ")
    ? "Key created"
    else
    If not instr($Userstring,$uservariable)
    $Userstring = "$Userstring,$uservariable"
    WriteValue($DPMkey,"ClientOwners", $Userstring, "REG_MULTI_SZ")
    EndIf
    Endif
    EndIf
    ==========================================================================
    The problem actually is that you still need to use an admin account to write on the registry, so ensure you configure it properly on the schedule task.
    In case you use a service account on the schedule task... the "$uservariable" will get populated with that account. As a work around to this... I changed it for the following line:
    =========================================================
    $uservariable = ReadValue("HKEY_LOCAL_MACHINE\SOFTWARE\Microsoft\Windows\CurrentVersion\Authentication\LogonUI", "LastLoggedOnSAMUser")
    =========================================================
    The only problem with that, is that key gets created/updated only if user gets logged phisically on that PC, but will not work for anyone connecting through RDP.

Maybe you are looking for